:100000001B29A801AA01A90001300828A900043071
:10001000A5002A082802031D0F28290827020430FA
:1000200003180130031902302505031D013017297B
:100030008030A100FE30BB200130BB207530A8000D
:100040003030E728A101A117B000FE30BB203008F6
:10005000BB28A401AB00AC01A01124080319A01512
:100060001030A3000301AB0DAC0D031801305C2070
:100070002308031D32280800A401AB00AC01A01125
:1000800024080319A0150530A3002730AA0010305A
:1000900055200330AA00E8305520AA0164305520CD
:1000A000AA010A3055202B085C28A9002C08A800BA
:1000B0002B08A700FB202708A700A3030319A01102
:1000C000240803196628230203186D282708031D36
:1000D000A011A0196D28303EBB280800AE00051005
:1000E00085108316051085100F30860583122E08A3
:1000F000A01898283E30A8008030E7203330AD00AB
:10010000AC201330A8008830E720AC206430E62013
:10011000AC206430E6202230AD00AC20283097209F
:100120000C30972006309720A0142E089828201411
:10013000AD00201CA6288510033C031CAB28AB2077
:100140000730A800D030E720031408002014FE3C3C
:100150000319B9288514201C201005140F308605BA
:100160002D08F03986040510AD0E2018AC28323069
:10017000E6202E081729A11B6E28080083169B0075
:1001800083161C141A089B0A172983169A001C153B
:1001900055309D00AA309D009C149C18CD281C1140
:1001A0009B0A172983178001840AFF3E031DD32869
:1001B0001729AA01A900FF30A907031CAA07031CDD
:1001C00017290330A800E530E720DB28A801F63E18
:1001D000A700A809031CF228FE300000A707031897
:1001E000ED28A7070000A80FEC2800002718F82822
:1001F0002718FA280800AC01AB011030AD00280D1B
:10020000AB0DAC0D2908AB022A08031C2A0FAC0267
:10021000031811292908AB072A0803182A0FAC076D
:100220000310A70DA80DAD0BFF282708172983136E
:10023000831203130800A00107309F008501860187
:10024000E33083168500FB30860081132030840064
:1002500060308312D320A03084005030D32020306F
:1002600084003030D2200515851505160130AA000E
:10027000F430DA20182054306E2072306E20613055
:100280006E206E306E2073306E2063306E207630BC
:100290006E2065306E2072306E2020306E204E3021
:1002A0006E204C306E2020306E2056306E202D3067
:1002B0006E2034306E208030A100C0302220773094
:1002C0006E206E206E202E306E2070306E206930D1
:1002D0006E2063306E2062306E2061306E2073308D
:1002E0006E2069306E2063306E202E306E206E30AE
:1002F0006E206C306E200730AA00D030DA20182033
:1003000049306E204E306E2053306E2054306E20B7
:1003100045306E204C306E203D306E204B306E20CC
:1003200065306E2075306E207A306E2065306E201C
:100330008030A100C03022205A306E2045306E201F
:100340004E306E2044306E203D306E2056306E2090
:1003500065306E2072306E2064306E2065306E2005
:1003600072306E2020306E2067306E2061306E203B
:100370006E206E306E200030BE20A6002608013AA6
:1003800001390319C512031DC516861C0E2A0A3031
:10039000D9200301C51A0130013A0319C512031D02
:1003A000C5168D302220A101C51EDD2952306E20D8
:1003B00043306E2035306E20E32952306E204330BA
:1003C0006E2036306E200618E729C122E32903018A
:1003D00006180130B200030186180130B205031976
:1003E000F329C122E7298030A100C5302220423004
:1003F0006E2065306E2076306E2065306E20733052
:100400006E2074306E2069306E2067306E2065304B
:100410006E206E306E2020306E20C5298618112A7D
:100420000E2A0030BE20A6002608C51A013C03197A
:10043000202A83169B0103018312C51A0130C520AF
:10044000C51E2D2A7F30BC001F30BD000130BE20EC
:10045000B8000230BE20C200372AFF30BC00FF3097
:10046000BD000330BE20B8000430BE20C2003808F2
:10047000B5004208BF00C51518207C22E52AB4014A
:10048000B30183108619831483184615831C461103
:1004900003018619013E4619013C03190130031D71
:1004A0000301B2003408A8003308A7000130AA00F5
:1004B00013300620B2050319612AB30A0319B40ADE
:1004C000482A3408013A133003193306031D692AF8
:1004D000102DC51C772A8310461D831483184615DA
:1004E000831C46110230A8007130E7207B2A0430BB
:1004F000A8004C30E72008008030A10022205330B3
:100500006E2079306E2073306E203A306E203F08B6
:100510003C2020306E206E208030A100C030222090
:1005200043306E206F306E206D306E203A306E207A
:1005300035083C2020306E206E20C51EB02A803049
:10054000A1008A3022200530A4003F082A208030F4
:10055000A100C83022200730A40035082A20C02A74
:100560008030A100883022200830A4003F082A20D3
:100570008030A100C83022200830A40035082A208D
:1005800008000A30D920BB0A33303B02031CD12AB1
:10059000BB01030105190130013A03190511031DBF
:1005A00005150800013006180301B2004308A70032
:1005B00000300120B2050319E42AC3030230D92018
:1005C0008618E32AE42AD22A08004515C51C4511DD
:1005D00005158515030186180130B20003010618C0
:1005E0000130B2050319F72AC830BE0045130301D4
:1005F00086180130B200030106180130B20503016C
:1006000086190130B2050319062BF72A86190A2B21
:10061000D82B172B0A30D920030186180130B200DD
:10062000030106180130B2050319172BE52A061835
:100630007D2B86181C2B1B2DC6104516C8303E027C
:10064000031D402BB430C400013006180301B20072
:100650004408A70000300120B2050319332B0530F0
:10066000D920C403242B013044020318402B03017A
:10067000C5190130013A0319C511031DC5154517E8
:10068000C51D542B851A4C2B3D08420203184A2BDA
:10069000C20A4B2BC201532B3C0838020318522BC1
:1006A000B80A532BB801652B851A5E2BC2080319B3
:1006B0005B2BC2035D2B3D08C200652BB8080319F4
:1006C000632BB803652B3C08B8003808B500420816
:1006D000BF007C22451F7C2B3E08C300D222C830BD
:1006E0003E02031D762BFA30C300D2220D303E02AB
:1006F000031C7C2B0C30BE02D72B8618D72B451E33
:10070000B92B4512C51E9F2B0130BE20A60026081E
:1007100038020319912B013083169B00831238088D
:10072000C5200230BE20A6002608420203199E2BD7
:10073000023083169B0083124208C520B92B033078
:10074000BE20A600260838020319AC2B03308316FE
:100750009B0083123808C5200430BE20A60026085E
:1007600042020319B92B043083169B0083124208FE
:10077000C520030146180130013A03194610031D34
:10078000461483104618831483180516831C05121B
:100790008618D72B0511C51ACF2B8F25D02B3825BE
:1007A00005150618D42B1B2D5230D920C82BE52A4D
:1007B000B401B301013086190301B2003408A80066
:1007C0003308A700FF30AA00DC300620B205031969
:1007D000ED2BB30A0319B40ADA2B4510C510B4087F
:1007E000031DF82B1E3033020318F82BE52A302C9A
:1007F000B408031DFF2B2D303302031C0B2CB4084F
:10080000031D0B2C3D30330203180B2C0830A800BD
:100810004D30E720302CB408031D122C5A3033021F
:10082000031C1F2CB408031D1F2C6F303302031848
:100830001F2C45140530A8000030E720302CB408E8
:10084000031D262C82303302031C2F2CB408031DF9
:100850002F2CB530330203182F2CC514302CE52A69
:100860003608B7004008C100B601C0010511C51C1B
:100870006C2C861D3C2C392C86193F2C3C2C861D5B
:10088000422C3F2C8619452C422C861D482C452C89
:100890000730A800D030E72083108619831483180E
:1008A0000516831C05120301051A013E8619013C39
:1008B000031D5B2C532C0430A8004C30E7203F2252
:1008C000C017461DC0133F224017461D40133F224C
:1008D000C016461DC012742C3F2283104619831483
:1008E00083180516831C05123F224016461D401230
:1008F0003F22C015461DC0113F224015461D401124
:100900003F22C014461DC0103F224014461D401017
:10091000C51C922C3F22B617461DB6133F22361730
:10092000461D36133F22B616461DB6123F22361616
:10093000461D36123F22B615461DB6113F2236150A
:10094000461D36113F22B614461DB6103F223614FE
:10095000461D3610451CAD2C361740084102031DBC
:100960000130B20036083702031D0130B204030122
:10097000C518013E4519013C031D0130B204013088
:10098000C6180301B20403190F2D1820451CD12CE1
:1009900052306E2043306E2035306E2058306E203D
:1009A000E02CC51CDA2C52306E2043306E203630DD
:1009B0006E20E02C52306E2043306E2035306E2099
:1009C00020306E2050306E2072306E206F306E20DE
:1009D00074306E206F306E2063306E206F306E206A
:1009E0006C306E200330AA00E830DA20C51CFA2CE7
:1009F000C512FB2CC5163608B5004008BF001820EC
:100A00007C22C6144008C2003608B8004614C51F30
:100A10004610C515C51C0E2DC5120F2DC516E52A8D
:100A2000051585110330AA00E830DA203708B60032
:100A30004108C000E52A182048306E2065306E203D
:100A400072306E2073306E2074306E2061306E20F4
:100A500072306E2074306E20013006180301B2002F
:100A6000013086180301B2040319372D2C2D1E29DD
:100A70007125381F7125381B6E2546187125461CB7
:100A80006E25421A7125421E6E25C2197125C21D9E
:100A90006E2542197125421D6E25C2187125C21C92
:100AA0006E2542187125421C6E25B81A7125B81E94
:100AB0006E25381A7125381E6E25B8197125B81D96
:100AC0006E2538197125381D6E25B8187125B81C8A
:100AD0006E2538187125381C6E2508007F25742571
:100AE000080074257F250800FF30BA0000000000D0
:100AF0000000000000000000BA0B762D0800203036
:100B0000B90000000F30BA00BA0B842D061505306D
:100B1000BA00BA0B892D0611B90B812D0800F325F7
:100B2000F325F325F325F325F325EC25EC25E9251D
:100B3000E625E625E625461CF325461CF325EC258F
:100B4000EC254618F3254618F325C21BE925C21FDC
:100B5000E625421BE925421FE625C21AE925C21EE9
:100B6000E625421AE925421EE625C219E925C21DDD
:100B7000E6254219E925421DE625C218E925C21CD1
:100B8000E6254218E925421CE625B81BE925B81FD1
:100B9000E625381BE925381FE625B81AE925B81ED1
:100BA000E625381AE925381EE625B819E925B81DC5
:100BB000E6253819E925381DE625B818E925B81CB9
:100BC000E6253818E925381CE6250800EC25F3252C
:100BD0000800F325EC250800E130BA000000000011
:100BE000BA0BEE2D08001030B90000000F30BA002B
:100BF000BA0BF82D06150530BA00BA0BFD2D0611FB
:080C0000B90BF52D0800032ECD
:02400E00023F6F
:0A42000000000000000000000000B4
:00000001FF
